:1030000039C000006EC000006CC000006AC0000043
:1030100068C0000066C0000064C0000062C000001C
:1030200060C000005EC000005CC00000E6C400009C
:1030300058C0000056C0000054C0000052C000003C
:1030400050C000004EC00000F2C200004AC00000A4
:1030500048C0000046C0000044C0000042C000005C
:1030600040C000003EC000003CC000003AC000006C
:1030700038C0000011241FBECFEFD2E0DEBFCDBFAD
:1030800004B603FE19C08091A0019091A101823481
:103090009C4D91F484B7877F84BF88E10FB6F89484
:1030A00080936000109260000FBE1092A1011092F8
:1030B000A001E0E0F0E0099511E0A0E0B1E0ECE86B
:1030C000FDE302C005900D92A239B107D9F721E0C6
:1030D000A2E9B1E001C01D92A03AB207E1F731D0F8
:1030E00053C68ECF84E08093E9008091E80085FD8F
:1030F0000EC08091E8008B778093E8008091E80013
:1031000082FDF3CF8EB38111F9CF80E008958091D5
:10311000F100089593E09093E9009091E80095FF05
:1031200003C08093F10008959091E8009E779093FA
:10313000E8009091E80090FDF4CF9EB39111F9CF93
:103140000895CF93DF9300D01F92CDB7DEB784B739
:10315000877F84BF88E10FB6F89480936000109257
:1031600060000FBE90E080E80FB6F8948093610095
:10317000909361000FBE11E015BF82E085BF2ED491
:1031800010936F0083E0809381007894A3E07A2EFF
:10319000B5E06B2E212C312C80910001882309F49D
:1031A0002FC284E08093E9008091E80082FF26C26C
:1031B00099DF982F853419F41092000107C088E830
:1031C000890F823010F0943521F48CDF8DE0A2DF7E
:1031D000EDC19035D9F39C34C9F3943721F484E4DC
:1031E00099DF80E0F4CF913611F489E5F0CF913486
:1031F00091F478DF082F76DF90E0880F991F202F59
:1032000030E0322F2227330F822B932BAA2797FDF2
:10321000A095BA2F9FC1903711F483E5D8CF93358D
:1032200071F47AE8E72E71E0F72EF70181917F01C2
:1032300071DFF1E9EF16F1E0FF06B9F7B7C1963596
:1032400021F481E367DF80E3C2CF933731F489E86B
:1032500061DF84E95FDF8EE1BACF9536A9F4E0E063
:10326000F0E070925700E89507B600FCFDCF609241
:103270005700E89507B600FCFDCFE058FF4FE11579
:1032800080E3F80771F7A2CF9C3651F42BDF8095CD
:1032900099E0E1E0F0E0082E90935700E89596CF92
:1032A000923721F489E0E1E0F0E010C0963419F49F
:1032B00089E0F1010BC09E3421F489E0E3E0F0E005
:1032C00005C0913539F489E0E2E0F0E080935700E1
:1032D00084917DCF923631F489E51CDF80E01ADFDE
:1032E00080E875CF923419F0973609F0CEC09983F3
:1032F000F9DEA82EB12CBA2CAA24F4DEA82AF2DE1C
:10330000082F8BEB800F9981823010F08FE35FCF15
:10331000973609F044C081E180935700E895450154
:10332000B12C8114910409F441C1C0909201D09054
:103330009301E0909401F09095010634B9F4EB2DDF
:10334000F0E0EC29FD298491E5DEBB2069F0F2E094
:10335000CF0ED11CE11CF11CC0929201D0929301BE
:10336000E0929401F0929501B12615C0D701C601F3
:10337000B695A79597958795F1D4CCDE82E0C80ED7
:10338000D11CE11CF11CC0929201D0929301E092F9
:103390009401F092950191E0891A9108C2CFC090F2
:1033A0009201D0909301E0909401F0909501063441
:1033B00029F0BB82AA82412C512C31C0F6017092B7
:1033C0005700E89507B600FCFDCFF3CF063479F53A
:1033D000552051F18090920190909301A09094011A
:1033E000B09095017FDE242D30E0382BF4010901E7
:1033F00010935700E8951124F2E08F0E911CA11C48
:10340000B11C8092920190929301A0929401B0928B
:10341000950151268A819B8101979B838A83EA814A
:10342000FB81EF2B99F626C05DDE482EF2CF5ADEE7
:10343000682F8091920190919301A0919401B09195
:103440009501B695A7959795879590D4809192010F
:1034500090919301A0919401B09195010296A11DC4
:10346000B11D8093920190939301A0939401B09326
:103470009501D0CF063409F0A9CEF601609257002D
:10348000E89507B600FCFDCFA1CE933469F4E09037
:103490009201F090930126DE90E0F7010C01109369
:1034A0005700E895112492CE9336F9F4C09092011A
:1034B000D0909301E0909401F090950113DEF60115
:1034C000E16090E00C0110935700E8951124F2E0C0
:1034D000CF0ED11CE11CF11CC0929201D09293013D
:1034E000E0929401F092950171CE9D3659F4E091ED
:1034F0009201F091930160925700E89507B600FCA5
:10350000FDCF64CE923551F4E0919201F091930198
:10351000E590F4908F2DFEDD8E2D59CE943419F563
:10352000E1DD682F8091920190919301A091940127
:10353000B0919501B695A7959795879517D48091E9
:10354000920190919301A0919401B09195010296FE
:10355000A11DB11D8093920190939301A0939401BA
:10356000B093950133CE9436F1F4C0909201D0908F
:103570009301E0909401F0909501D701C601B695B2
:10358000A79597958795EAD3C5DD82E0C80ED11C33
:10359000E11CF11CC0929201D0929301E09294013F
:1035A000F092950103C09B3109F0B0CE7092E90012
:1035B0009091E8008091E8008E778093E80095FD77
:1035C00011C08091E80080FD04C08EB38111F9CF55
:1035D00015C08091E8008E778093E80003C08EB319
:1035E000882361F08091E80080FFF9CF94E0909308
:1035F000E9008091E8008B778093E80094D3CCCDEC
:103600008091E00081608093E00082E49CED9093E3
:10361000A1018093A0012CE088E190E00FB6F8941E
:10362000A895809360000FBE20936000FFCF1F928B
:103630000F920FB60F9211240F900FBE0F901F9094
:10364000189542E061EC82E062D142E161E883E0FA
:103650005ED142E160E884E05AC180919801982FE0
:103660009F77913299F590919901913229F0923298
:1036700029F1903259F510C0813A41F58091E80066
:10368000877F8093E80067E070E081E091E0A4D05C
:103690008091E8008B770FC08132C1F48091E800FF
:1036A000877F8093E80067E070E081E091E0F5D0EB
:1036B0008091E8008E778093E8000895813231F49C
:1036C0008091E800877F8093E80035C10895292F15
:1036D00030E02230310539F02330310549F0213016
:1036E000310561F410C08EE390E02AE331E01EC0A2
:1036F000882371F0813089F08230A1F080E090E081
:1037000020E030E013C082E190E028E731E00EC015
:1037100084E090E026E331E009C088E190E02CE10C
:1037200031E004C082E190E028E031E0FA01318329
:103730002083089507B600FCFDCFF999FECF23E062
:10374000FB0120935700E89507B600FCFDCF81E10F
:1037500080935700E895089507B600FCFDCFF999CE
:10376000FECF25E0FB0120935700E89507B600FC4B
:10377000FDCF81E180935700E895089507B600FCDE
:10378000FDCFF999FECF21E0FB010A0120935700FC
:10379000E8951124089521E2FC01209357008491BB
:1037A000089529E0FC012093570084910895E1E0F9
:1037B000F0E089E0809357008491089507B600FCFB
:1037C000FDCFF999FECF809599E0E1E0F0E0082E79
:1037D00090935700E895089520919E0130919F01A4
:1037E0002617370748F06115710539F42091E80074
:1037F0002E772093E80001C0B90120E06115710522
:10380000C9F13EB3332309F442C0353009F441C055
:103810003091E80033FD3FC03091E80032FF06C030
:103820008091E80082FF29C080E008953091E8008F
:1038300030FFE4CF2091F20030E0FC01281B390B6F
:10384000CF01820F931F6115710549F088309105F2
:1038500030F481918093F10061507109F1CF21E042
:10386000089709F020E08091E8008E778093E800C7
:10387000CF01C4CF2111C5CFD3CF8EB3882339F068
:10388000853039F08091E80083FFCACF04C082E020
:10389000089583E0089581E008956115710529F484
:1038A0002091E8002B772093E8006115710511F154
:1038B0002EB3222341F1253041F12091E80023FD70
:1038C0001EC02091E80022FFF3CFFC01CF01209120
:1038D000F200222329F38091F1008193CF016150FE
:1038E00071096115710591F7DBCF8EB3882359F00B
:1038F000853059F08091E80080FFF7CF02C081E069
:10390000089580E0089582E0089583E008958F701F
:103910008093E900EBEEF0E0808181608083EDEE42
:10392000F0E010826093EC0040838091EE00881FED
:103930008827881F08958091980187FD05C0809190
:10394000E80080FF0DC010C08091E80082FD04C037
:103950008EB38111F9CF08958091E8008B7707C06D
:103960008EB38111ECCF08958091E8008E7780931B
:10397000E80008953CD03ED08091D8008F778093A6
:10398000D8008091D80080688093D8008091D800BA
:103990008F7D8093D80084E089BD86E089BD09B41D
:1039A00000FEFDCF1EBA1092960142E060E080E07A
:1039B000AEDF8091E1008E7F8093E1008091E20094
:1039C00081608093E2008091E20088608093E20051
:1039D0008091E0008E7F8093E0000895E3E6F0E0C0
:1039E00080818E7F808381E080939701C3CF109286
:1039F000E20008951092E10008951F920F920FB611
:103A00000F9211242F933F934F935F936F937F9364
:103A10008F939F93AF93BF93EF93FF938091E100B8
:103A200080FF16C08091E20080FF12C08091E2000A
:103A30008E7F8093E2008091E20080618093E200BB
:103A40008091D80080628093D80019BC1EBA6AD1D8
:103A50008091E10084FF2EC08091E20084FF2AC0A3
:103A600084E089BD86E089BD09B400FEFDCF809168
:103A7000D8008F7D8093D8008091E1008F7E809365
:103A8000E1008091E2008F7E8093E2008091E2006D
:103A900081608093E20080919601882311F084E098
:103AA00007C08091E30087FF02C083E001C081E08E
:103AB0008EBB38D18091E10083FF21C08091E2006C
:103AC00083FF1DC08091E100877F8093E10082E049
:103AD0008EBB109296018091E1008E7F8093E10071
:103AE0008091E2008E7F8093E2008091E20080610D
:103AF0008093E20042E060E080E009DF13D1FF91B3
:103B0000EF91BF91AF919F918F917F916F915F9155
:103B10004F913F912F910F900FBE0F901F901895CE
:103B20001F93CF93DF9300D0CDB7DEB7E8E9F1E084
:103B30008091F100819381E0E03AF807C9F78DDDCB
:103B40008091E80083FFDAC09091980180919901FB
:103B5000853009F465C030F4813059F168F0833064
:103B600041F1CCC0883009F49CC0893009F4ABC065
:103B7000863009F0C3C075C0903881F0923809F0E2
:103B8000BDC080919C018F708093E9009091EB0003
:103B900095FB992790F91092E90001C090E080917F
:103BA000E800877F8093E8009093F1001092F10085
:103BB00083C0292F2D7F09F0A1C0923009F09EC04B
:103BC00090919A01911126C020919C012F7009F4C7
:103BD00095C02093E9009091EB0090FF1BC08330CB
:103BE00021F48091EB00806213C08091EB00806132
:103BF0008093EB0081E090E0022E01C0880F0A94D0
:103C0000EAF78093EA001092EA008091EB00886066
:103C10008093EB001092E9008091E800877F4FC00D
:103C200091116CC010919A011F778091E300807808
:103C3000812B8093E3008091E800877F8093E800E8
:103C40007ADE8091E80080FFFCCF8091E3008068FD
:103C50008093E300112311F083E001C082E08EBB6A
:103C60004DC09058923008F049C0AE014F5F5F4F91
:103C700060919C0180919A0190919B0128DD0097B1
:103C800009F43CC02091E800277F2093E800BC01A4
:103C900089819A81A1DD8091E8008B778093E8008B
:103CA0002DC0903859F58091E800877F8093E80017
:103CB000809196018093F1008091E8008E77809347
:103CC000E80039DE1BC0911119C090919A01923021
:103CD000A8F48091E800877F8093E8009093960194
:103CE0002ADE80919601811104C08091E30087FF54
:103CF00002C084E001C081E08EBBA3DC8091E800BB
:103D000083FF0AC08091E800877F8093E80080915C
:103D1000EB0080628093EB000F900F90DF91CF91CA
:103D20001F9108950895CF938EB38823A9F08091B1
:103D3000E9008F709091EC0090FF02C090E801C004
:103D400090E0C92FC82B1092E9008091E80083FD14
:103D5000E7DECF70C093E900CF910895F999FECFC7
:103D600092BD81BDF89A992780B50895262FF999BB
:103D7000FECF1FBA92BD81BD20BD0FB6F894FA9A4E
:0C3D8000F99A0FBE01960895F894FFCF49
:103D8C00010000000000000812034C005500460022
:103D9C00410020004300440043000000180344008D
:103DAC00650061006E002000430061006D0065003D
:103DBC007200610000000403090409023E000201C4
:103DCC0000803209040000010202010005240010E9
:103DDC0001042402020524060001070582030800E1
:103DEC00FF09040100020A0000000705040210008C
:103DFC0005070583021000051201100102000008DE
:103E0C00EB034A200001010200014C55464143449A
:023E1C00430061
:103FA000C9CBDACBEBCBF7CBFCCB01CC07CC08955C
:083FB000089508950895089595
:103FE000DFCFDFCFDFCFDFCFDFCFDFCFDFCFDFCF61
:083FF000DFCFDFCFDFCFDFCF11
:083FF8000030000000DFFBDCDB
:0400000300003000C9
:00000001FF
